:10000000AD28A30038088400360928208413A308EB
:100010000319A828F030A50022088038A400F03089
:10002000A5030319A5000319A3030319A828182879
:100030002B20030120183608A21F3608A208031936
:100040000301A40F252880060C28262800000F286D
:1000500084178005A828210820040319A00A8030ED
:10006000201AA1062019A106A018A106210DA00D95
:10007000A10DA82883169B001C141A08A828831613
:100080009A001C1555309D00AA309D009C149C18A8
:1000900047281C11A828A301A200FF30A207031CB7
:1000A000A307031CA8280330A100DF3059204D28E6
:1000B000A101E83EA000A109FC30031C6228A007B2
:1000C00003185F28A0076400A10F5F282018682884
:1000D000A01C6C2800006C280800A301A2000230BC
:1000E0007C28A20003307C28A20001307C28A200DA
:1000F00006307C28A2000530A80023082102031D39
:10010000832822082002043003180130031902302A
:100110002805031DFF30A828A501A4011030A60062
:10012000210DA40DA50D2208A4022308031C230FF2
:10013000A5020318A2282208A40723080318230FE6
:10014000A5070310A00DA10DA60B90282008A82834
:10015000831303138312640008008316FF239000A7
:100160008312850107309900831611308500103005
:100170009500811311309F00831281309F00C401CC
:10018000C201C3016400051AC6285721F2213E08A6
:10019000A0003F08A100A30100307A20031DD12850
:1001A000C22801303A20C5003E08A0003F08A10047
:1001B00045086D20031DDD285429F2213E08A000CA
:1001C0003F08A100A30100307A20031DE828C228BF
:1001D00002303A20C6003E08A0003F08A1004608B1
:1001E0006D20031DF4285429F2213E08A0003F0889
:1001F000A100A30100307A20031DFF28C22803308C
:100200003A20C7003E08A0003F08A10047086D2023
:10021000031D0B295429F2213E08A0003F08A1002C
:10022000A30100307A20031D1629C22804303A2089
:10023000C8003E08A0003F08A10048086D20031D2B
:100240002229542985168316851283128514831654
:1002500085108312C4010511831605110530831220
:10026000B8002030B6006430A2000A300120783097
:10027000A2000A3001206430A2000A300120783048
:10028000A2000A3001206430A200143001200B309B
:10029000A300B8304C208510831685108312851278
:1002A000831685128312C228C201C301C228BA0173
:1002B000BB013A08A0003B08A1003A30A3009830E7
:1002C0007420031D6B296400051E67290800BA0A03
:1002D0000319BB0F5929C4016400051D74290511B8
:1002E0008316051183120800851683168512831262
:1002F000F2213E08A0003F08A100A30100307A20AF
:10030000031D8729851283168512831208003E0873
:10031000C500F2213E08A0003F08A100A301003063
:100320007A20031D982985128316851283120800EE
:100330003E08C600F2213E08A0003F08A100A3012C
:1003400000307A20031DA929851283168512831295
:1003500008003E08C700F2213E08A0003F08A100A7
:10036000A30100307A20031DBA2985128316851255
:10037000831208003E08C800831601309B008312D8
:1003800045083F20831602309B00831246083F2019
:10039000831603309B00831247083F2083160430E6
:1003A0009B00831248083F200530B8002030B6007B
:1003B0006430A2000A3001206930A2000A30012016
:1003C0006E30A2000A3001207330A2000A300120F2
:1003D0007830A20014300120851283168512831212
:1003E000C4010800FE224008A0004108A100A301AA
:1003F00028307120031DFD29B62A0130A100F430F8
:100400005920FE224008BE004108BF000130BA005A
:10041000BB013A08A0003B08A100A30109307420E9
:10042000031D442AFE224008A0004108A100A301A8
:1004300028307120031D1D2AB62A3E08A0003F085F
:10044000A1003A08A2003B08A3008C20B2002108BA
:10045000B3001E30B2020030031C013EB30240085C
:10046000A0004108A1003308A30032087120031D39
:100470003A2AB62A4008BE0741080318013EBF07C2
:10048000BA0A0319BB0F092A3E08A0003F08A100C1
:100490000A30A200A3018C20B2002108B30046302C
:1004A000B2070318B30A3208A0003308A100553080
:1004B000A200A3018C20BE002108BF000530B800B7
:1004C0002030B6006E303E07B2003F080318013EF0
:1004D000B3003208A2000A30012085168316851267
:1004E0008312BA01BB013A08A0003B08A100A30196
:1004F00014307420031D8B2AFE224008A0004108FE
:10050000A100A30128307720031D872A7C2ABA0A7C
:100510000319BB0F732ABC01BD01C40A6400283053
:100520004402031CB12A0530B8002030B6006E30FA
:10053000A200053001207D30A200053001206E3080
:10054000A200053001207D30A200053001206E3070
:10055000A2000530012005158316051183122730EE
:10056000C400851283168512831208003C08A0007F
:100570003D08A100FD30A300E8307720031DFA2AD2
:10058000BC01BD01BE01BF010530B8002030B6007E
:100590007D30A2000130012085128316851283125E
:1005A000C20A0319C30A4208A0004308A10001308F
:1005B000A300C2307A20031DE82A05118316051115
:1005C0006400053083124402031CE82A0430C4028C
:1005D0004208A0004308A1001330A3008830772010
:1005E000031DF92AC201C301C401051183160511B7
:1005F00083120800BC0A0319BD0AF2299F14640083
:100600009F1C032BFF2A1E08C10083161E0883129D
:08061000C000080063000A2B82
:02400E00C43FAD
:00000001FF
